:020000040000FA
:020000000428D2
:08000800FF30A1003D2083162A
:1000100001309F00831207309900FF3049202112E0
:100020004820A112472022124320A2124220221669
:100030004320851C222812305520221243200230F2
:10004000552028280C3055202212432008305520F6
:10005000A2164220051D332812305520A21242203C
:100060000230552039280C305520A2124220083089
:10007000552010304E2017283C288316FF2390006F
:1000800083120800442844282208850008004B28D1
:100090004B28A1004B28210865000800A300230875
:1000A000A4000A30A50001305C28A3002308A400A6
:1000B0000130A50001305C28A600FF30A70025080C
:1000C000A9002408A8001730270703186428A80BE4
:0C00D0006328A90B6128A60B5F2808001C
:02400E0084111B
:00000001FF
